S123B8007EBE507EBEA87EBDA77EBDB47EBEBB7EBDD97EBE4A7EBE480A0D4D433638373052
S123B820312050524F4752414D4D4552204F4E204C494E450A0D0A0D040D0A4C4F41442029
S123B840434F4D504C45544544200A0D4C415354204144445245535320424C4F434B204CBF
S123B8604F41444544203D20040A0D0A0D50524F4752414D494E472041424F525445440A97
S123B8800D040808080808040A0D54484520544553542057494C4C20434C45415220544874
S123B8A0452050524F4752414D4D45522052414D0D0A0D0A202020202020205459504520B3
S123B8C02D592D20544F20434F4E54494E554520040A0D4D454D4F525920434F4E54454E6E
S123B8E0545320554E4348414E4745440A0D040A0D4C4F4144204552524F52202D2D204317
S123B9004845434B53554D204D49534D41544348200A0D040A0D4C4F4144204552524F5281
S123B920202D2D2052414D2044415441204D49534D41544348200A0D040A0D4C4F41442047
S123B9404552524F52202D2D2041444452455353204F5554204F462052414E4745200A0D28
S123B960040A0D0A0D4C4F41442041424F525445442C204E4F204441544120444F574E4C89
S123B9804F414445440A0D040A0D4D433638373031204953204552415345440A0D040A0DBC
S123B9A050524F4752414D4D494E4720040D0A0D0A50524F4752414D4D494E4720434F4DAC
S123B9C0504C4554450A0D0A0D040A0D434F5059494E47204550524F4D20544F2052414D21
S123B9E0200A0D0A0D04564552494659494E47204D4336383730310A0D044D433638373008
S123BA0031204E4F54204552415345440A0D04454E544552202D592D20544F204F56455281
S123BA2050524F4752414D0A0D4F5220414E59204F5448455220434841522E20544F2045F4
S123BA404E4420044550524F4D20444F4553204E4F54204D415443482052414D0A0D46491A
S123BA60525354204144445245535320494E204552524F52203D20040A0D0A0D4144445278
S123BA80455353204F5554204F462052414E47450A0D040A0D040A0D4D454D4F52592054C3
S123BAA0455354205041535345440A0D040A0D4D454D4F52592054455354204641494C45CA
S123BAC0440A0D044D43363837303120434F4E54454E54532056455249464945440A0D0456
S123BAE00D0A5331040D0A3E040A0D5339040D0A2404504F5254203120424144200A0D04AC
S123BB00504F5254203120504153534544200A0D04CEBA93BDBDD939BDBEC6CEB888BDBD00
S123BB20D9BDBEA881592709CEB8D1BDBDD97EBE7D8600C601CE8800A700084C81FF260252
S123BB401B5C8C900026F18600C601CE8800A100262E084C81FF26021B5C8C900026EF8675
S123BB60AA8D22261B86558D1C261586FF8D16260F86008D102609CEBA96BDBDD97EBE7D8F
S123BB80CEBAAD20F5CE8800A700088C900026F8CE8800A1002606088C900026F639BDBE01
S123BBA0C6BDBBC52705BDBBE62609BDBBF2BDBC657EBE7DCEB869BDBDD97EBE7DBDBEC688
S123BBC08D037EBE7DCEF800A60026118CFFFF27030820F4CEB988BDBDD9860039CEB9FA03
S123BBE0BDBDD986FF39CEBA0FBDBDD9BDBEA8815939CEB99EBDBDD9C6FED714CE8FFFDFAE
S123BC0082CE7797DF90CEF800DF8ECE88003C968F260ECE008EBDBE48CEB882BDBDD93883
S123BC203CA6008100271BDE8EA70086FC9714DC90D3097F0008DD0B8640950827FC86FE5A
S123BC409714DE8E08DF8E38088C8FFF23C086FF9714CEB9ADBDBDD939BDBEC686FF9714B6
S123BC608D037EBE7DCEB9E6BDBDD9CEF800DF8ECE88003CA600DE8EE60011261108DF8E3D
S123BC8038088C8FFF23ECCEBAC4BDBDD939CEBA44BDBDD9CE008EBDBE48BDBB113839BD6A
S123BCA0BEC6CEB9CABDBDD9CE8800DF8E86FF9714CEF800A600083CDE8EA70008DF8EFC31
S123BCC007D0D3097F0008DD0B8640950827FC388C000026DFBDBC657EBE7D86FF97877F36
S123BCE00092BDBEA8815326F9BDBEA881392756813126EE96928A0897927F0086BDBDB462
S123BD008002978CBDBDA796872709DC84C39000DD84DE848C8800255E8C90012459BDBDEB
S123BD20B47A008C2709A700A10026110820E57C008627AE96928A0497927EBCE296928A05
S123BD400297927EBCE2BDBEA8810D26F9BDBB1196928407262A969285082712CEB839BDD2
S123BD60BDD9CE0084BDBE48BDBB117EBE7DCEB961BDBDD97EBE7D96928A0197927EBCE2E6
S123BD80969285012706CEB939BDBDD9969285022706CEB914BDBDD9969285042706CEB883
S123BDA0EFBDBDD97EBE7DBDBDB49784BDBDB49785DE84398D7148484848168D6A1B16DB1F
S123BDC086D7863944444444840F8B30813923028B077EBEBBBDBEBB08A600810426F639BF
S123BDE07EBE7D86FF9714BDBDA7CEBAEE8DEACE00848D54DE848D528D52BDBEA88120270A
S123BE00F9810D27DB815E2704812C26060909DF8420D7DF84813025D1814622CD8D0BBD31
S123BE20BDB609A70020C3BDBEA880302B0F81092F0A81112B0781162E03800739203EA6D8
S123BE40008D81A6000820808DF58DF38620206B8E00FF86FF9714867F97008606D602C4CE
S123BE6080260286059710860A971196119612CE0FFF09010126FBCEB818BDBDD98E00FFD7
S123BE8086FF97147F0087CEBAE5BDBDD9BDBEA8CEBF8DA1002607BDBE4CEE016E00080869
S123BEA0088CBFAE26ED20D5379611848027FA9612847F81602D058020200137D611C420F1
S123BEC027FA97133339BDBEA8810D2601397EBE7DBDBE4CBDBDA73CBDBEC6BDBB1138BD7A
S123BEE0BF586E008D09CEBAE9BDBDD97EBE7DBDBE4CBDBDA7BDBF58DF88BDBE4CBDBDA79B
S123BF00BDBF58DF82BDBEA8810D27037EBE7D96839089D682D288260481102502860F8B6E
S123BF2004978C8003978ACEBAE0BDBDD95FCE008C8D20CE00888D1B8D19DE888D157A00EB
S123BF408A26F9DF885337308D0933DE88099C8226BD39EB007EBE3F8C900025068CF80070
S123BF602507398C8800250139CEBA78BDBDD97EBE7D867F9700CEBAF29702910226084A1F
S123BF8081FF26F5CEBB00BDBDD97EBE7D50BB9E4DBDE345BBBD56BC5944BCDB54BB184A63
S111BFA0BED152BC9F43BF7255BEE44CBCDF01
S113BFF0BE50BE50BE50BE50BE50BE50BE50BE50CD
S9030000FC
